:100000000E28FF3FFF3FFF3F8B13CC000308830107
:10001000CD000A08CE000408CF000D2F5F308316F4
:1000200003138F00831603178801831603178901B2
:1000300083160313203085000F30860000308700C0
:1000400083120313AF255C248C225C2483120317D4
:1000500000308D00831603178C130C1483120317C2
:100060000C080313D8008312031701308D00831688
:1000700003178C130C14831203170C080313D900F5
:100080008312031702308D00831603178C130C1490
:10009000831203170C080313DA00831203170430CA
:1000A0008D00831603178C130C14831203170C088E
:1000B0000313E1008312031705308D008316031725
:1000C0008C130C14831203170C080313E000601345
:1000D0008312031703308D00831603178C130C143F
:1000E000831203170C080313DE005F14DF17DE1AF8
:1000F000F528FE288A26D4005C24DF135F145418E8
:100100008B28D418AA285419C828D419E628541AB8
:100110001A295F10C229541BD80A541FD803580843
:10012000403C0319D8035808073C0319D80A611347
:100130000A168A1100200A128A11902483120317CA
:1001400000308D00831203135808831203178C00AC
:100150008022C229541BD90A541FD90359081A3CBA
:100160000319D9035908053C0319D90A0A128A153B
:1001700000200A128A1190248312031701308D0087
:10018000831203135908831203178C008022C2299B
:10019000541BDA0A541FDA035A080B3C0319DA031A
:1001A0005A08013C0319DA0A0A128A153F210A1279
:1001B0008A1190248312031702308D0083120313D7
:1001C0005A08831203178C008022C229541BDE0AAE
:1001D000541FDE035E08393C0319DE035E08063C4B
:1001E0000319DE0ADE1AF528FE281F30DC005E083F
:1001F000DB00DB09DB135B13DB1206291F30DB009E
:100200005E08DC00DC135C13DC120629DF1B982877
:100210000A128A15BF210A128A1190248312031729
:1002200003308D00831203135E08831203178C00C2
:100230008022C229541B1D292029D41A31292A2998
:10024000D41A23293829DE22E1156111E110611049
:100250009325C229E822E1116115E114611093256B
:10026000C229F222E1116115E11461149325C2291A
:10027000B421E20062183D29B02954238B25640083
:100280008A26D400D41B3F29541E3F29541B4929D8
:100290004C29D41A93296E29D41A4F293F29962321
:1002A0008125932564008A26D400D41B5229541E2C
:1002B0005229541B5C295F29D41A52296829D41A5F
:1002C00062295229E113E11261125C249325C229AB
:1002D000E113E11661125C249325C229D8238125FC
:1002E000932564008A26D400D41B7129541E7129D9
:1002F000541B7B297E29D41A8D298729D41A812958
:100300007129E113E11261165C249325C229E113DE
:10031000E11661165C249325C229E117E1166116E6
:100320005C249325C2291A2481259325C2296400BF
:100330008A26D400D41B9629541E9629541BA12921
:10034000A429D41AAD29AA29D41AA72996295C244C
:100350009325C2295C249325C2295C249325C229B4
:10036000FC2261179325C2290A30D6006430D500DB
:100370008A26D400D41B0034D50BB829D60BB62955
:10038000640001345F1CEA290830D3006008D20001
:100390001E270930D3006108D2001E270030D30089
:1003A0005808D2001E270130D3005B08D2001E2758
:1003B0000230D3005C08D2001E270330D300590856
:1003C000D2001E270430D3005A08D2001E278125F0
:1003D0006F257A2886128316031385168316031752
:1003E000881683160313861683160317891683123D
:1003F00003138B258B258316031300309F00831274
:10040000031311309F008B259F149F18052A831218
:1004100003131E08E300831203130430E3077E2452
:100420000A168A1500200A128A117008A0007108A5
:10043000A1007208A2007308A3007408A400750844
:10044000A5007608A6007708A7007808A800790814
:10045000A9007A08AA007B08AB007C08AC007D08E4
:10046000AD007E08AE007F08AF0083160313003096
:100470009F008316031386168316031789168312AB
:10048000031335309F008B259F149F18452A831234
:1004900003131E08E300831603178801831603174E
:1004A0008901831603138612831203130430E307B2
:1004B0007E240A168A1500200A128A117008B000DC
:1004C0007108B1007208B2007308B3007408B40078
:1004D0007508B5007608B6007708B7007808B80048
:1004E0007908B9007A08BA007B08BB007C08BC0018
:1004F0007D08BD007E08BE007F08BF0090247A28DA
:10050000831603178C130C1555308D00AA308D00FF
:100510008C148312031308006530A8006C30A90006
:100520007730AA006530AB006230AC002E30AD00F1
:100530006330AE007A30AF00FF30B00081259024E8
:10054000FF30B10081259024FF30B2008125902436
:10055000FF30B30081259024FF30B4008125902422
:10056000FF30B50081259024FF30B600812590240E
:10057000FF30B70081259024FF30B80081259024FA
:10058000FF30B90081259024FF30BA0081259024E6
:10059000FF30BB0081259024FF30BC0081259024D2
:1005A000FF30BD0081259024FF30BE0081259024BE
:1005B000FF30BF0081259024902408002830A5003A
:1005C0004130A6002930A7007E30A8009024080002
:1005D0002830A5004230A6002930A7007E30A800B0
:1005E000902408002830A5004330A6002930A70039
:1005F0007E30A800902408002830A5004D30A600C9
:100600005530A7005430A8004530A9002930AA0071
:100610009024812581258A26D400D41B08006830C7
:10062000B0006F30B1006C30B2006430B300FE3007
:10063000B4009024812581258A26D400D41B08008B
:100640006630B5006F30B6007230B700FE30B800CB
:100650009024812581258A26D400D41B08006D3082
:10066000B9006530BA006E30BB007530BC00902414
:10067000812581258A26D400D41B08002E30BD0098
:100680009024812581258A26D400D41B08002E3091
:10069000BE009024812581258A26D400D41B080021
:1006A0002E30BF00902408004130A000FE30A10091
:1006B0006D30A2006F30A3006E30A4006F30A50033
:1006C000FE30A600FE30A700FE30A800FE30A900D4
:1006D0004330AA00FE30AB006230AC006130AD00A8
:1006E0006330AE006B30AF004230B000FE30B1007E
:1006F0007330B2007430B3006530B4007230B500AE
:100700006530B6006F30B700FE30B800FE30B9007B
:10071000FE30BA00FE30BB00FE30BC00FE30BD0033
:10072000FE30BE00FE30BF00902408004130A00023
:10073000FE30A1006E30A2006F30A3007230A40022
:100740006D30A5006130A6006C30A700FE30A80017
:100750006D30A9006F30AA006E30AB006F30AC0076
:10076000FE30AD00FE30AE00FE30AF004230B000D3
:10077000FE30B1007030B2007330B3006530B400A9
:100780007530B5006430B6006F30B700FE30B80089
:100790007330B9007430BA006530BB007230BC00F1
:1007A0006530BD006F30BE00FE30BF0090240800F1
:1007B0007330A0007030A1006130A2007430A3003B
:1007C0006930A4006130A5006C30A600FE30A7009F
:1007D0006530A8006630A9006630AA006530AB001D
:1007E0006330AC007430AD00FE30AE00FE30AF00C0
:1007F0004130B000FE30B1003030B2002530B300DF
:10080000FE30B4004230B500FE30B6003330B700E1
:100810003030B8002530B900FE30BA004330BB009C
:10082000FE30BC003530BD003230BE002530BF0088
:10083000902408004130A000FE30A100FF30A2004B
:10084000FF30A300FF30A400FE30A500FE30A6005C
:10085000FE30A700FE30A800FE30A9004330AA00F9
:10086000FE30AB006930AC006E30AD006630AE00DB
:100870006F30AF004230B000FE30B100B030B20097
:10088000B030B300B030B400FE30B500FE30B6007A
:10089000FE30B700FE30B800FE30B900FE30BA00BE
:1008A000FE30BB00FE30BC00FE30BD00FE30BE009E
:1008B000FE30BF0090240800FE30A000A100A2007E
:1008C000A300A400A500A600A700A800A900AA00F4
:1008D000AB00AC00AD00AE00AF00B000B100B200A4
:1008E000B300B400B500B600B700B800B900BA0054
:1008F000BB00BC00BD00BE00BF000800FE30F00021
:10090000F100F200F300F400F500F600F700F80043
:10091000F900FA00FB00FC00FD00FE00FF000800EB
:100920000713803051250717200851250713813000
:100930005125071721085125071382305125071724
:100940002208512507138330512507172308512505
:1009500007138430512507172408512507138530C4
:1009600051250717250851250713863051250717EC
:1009700026085125071387305125071727085125C9
:100980000713883051250717280851250713893088
:10099000512507172908512507138A3051250717B4
:1009A0002A08512507138B30512507172B0851258D
:1009B00007138C30512507172C08512507138D304C
:1009C000512507172D08512507138E30512507177C
:1009D0002E08512507138F30512507172F08512551
:1009E0000713C03051250717300851250713C130B0
:1009F00051250717310851250713C2305125071714
:100A0000320851250713C3305125071733085125E4
:100A10000713C43051250717340851250713C53073
:100A200051250717350851250713C63051250717DB
:100A3000360851250713C7305125071737085125A8
:100A40000713C83051250717380851250713C93037
:100A500051250717390851250713CA3051250717A3
:100A60003A0851250713CB30512507173B0851256C
:100A70000713CC30512507173C0851250713CD30FB
:100A8000512507173D0851250713CE30512507176B
:100A90003E0851250713CF30512507173F08512530
:100AA0000800D10087100710871305128511051162
:100AB0008510051051188714D1180714511987177C
:100AC000D1190516511A8515D11A0515511B851412
:100AD000D11B05140715912507118B25080014302B
:100AE000C2001430C1006430C00064008A26D40003
:100AF000D41F0800C00B7A2DC10B732DC20B712DB2
:100B000008001430D600FF30D500D50B852DD60B4C
:100B1000832D640008006430D700D70B8D2D64004E
:100B200008000000080064008A26D400D41F932D1A
:100B30008312031704308D0083120313610883129C
:100B400003178C0080228312031705308D00831257
:100B500003136008831203178C008022080081258C
:100B60008711071301305125071302305125071350
:100B70000630512507130C30512507131430512529
:100B8000071338305125071340305125071703301C
:100B90005125071703305125071703305125071733
:100BA000033051250717033051250717033051250E
:100BB0000717033051250717033051250717103049
:100BC00051250713003051250713483051250717C9
:100BD000183051250717183051250717183051259F
:100BE00007171830512507171830512507171830E7
:100BF00051250717183051250717183051250717A9
:100C0000103051250713003051250713503051255E
:100C100007171030512507171030512507171030CE
:100C20005125071710305125071710305125071788
:100C30001030512507171030512507171030512556
:100C4000071710305125071300305125071358306E
:100C5000512507171C30512507171C305125071740
:100C60001C30512507171C30512507171C30512502
:100C700007171C30512507171C30512507171C304A
:100C80005125071710305125071300305125071340
:100C90006030512507171E30512507171E3051258A
:100CA00007171E30512507171E30512507171E3014
:100CB000512507171E30512507171E3051250717DC
:100CC0001E305125071710305125071300305125CC
:100CD00007136830512507170F30512507170F30BC
:100CE000512507170F30512507170F3051250717CA
:100CF0000F30512507170F30512507170F30512599
:100D000007170F30512507171030512507130030F2
:100D10005125080006128612061386138B25061C21
:100D2000982E861CB22E061DCB2E861DE42E8034F6
:100D300006128616061786178B25061CFD2E06162C
:100D4000861206178617061CFE2E06168616061332
:100D50008617061CFF2E0616861606178613061C17
:100D6000002F80340612861606178617861C012F60
:100D70000616861206178617861C022F061686167A
:100D800006138617861C032F06168616061786136B
:100D9000861C042F80340612861606178617061D39
:100DA000052F0616861206178617061D062F06162D
:100DB000861606138617061D072F061686160617B3
:100DC0008613061D082F803406128616061786170E
:100DD000861D092F0616861206178617861D0A2FEE
:100DE0000616861606138617861D0B2F0616861600
:100DF00006178613861D0C2F803442344834703415
:100E00008034023408345034803441344434103453
:100E100080340134043430348034831600308B0045
:100E20008B1520308C00831283014F0884004E08FC
:100E30008A004D088300CC0E4C0E09000716871659
:100E40000000000000000000000087120000000009
:100E50000000071200000000000087169B27871281
:100E60009B2787129B2787129B2787129B27871216
:100E70009B2787129B2787129B2788278712D31BC4
:100E800087169B278712531B87169B278712D31A17
:100E900087169B278712531A87169B278712D31909
:100EA00087169B278712531987169B278712D318FB
:100EB00087169B278712531887169B278827871228
:100EC000D21B87169B278712521B87169B278712D8
:100ED000D21A87169B278712521A87169B278712CA
:100EE000D21987169B278712521987169B278712BC
:100EF000D21887169B278712521887169B27882798
:100F0000000000000000071600000000871608001F
:100F10008316871683129B27871E8C2F00000000E4
:100F20000000000000000000000000000000831628
:100F300087128312080000000716000064000000FA
:100F4000071200000800FF3FFF3FFF3FFF3FFF3F4A
:100F5000FF3FFF3FFF3FFF3FFF3FFF3FFF3FFF3FA1
:100F6000FF3FFF3FFF3FFF3FFF3FFF3FFF3FFF3F91
:100F7000FF3FFF3FFF3FFF3FFF3FFF3FFF3FFF3F81
:100F8000FF3FFF3FFF3FFF3FFF3FFF3FFF3FFF3F71
:100F9000FF3FFF3FFF3FFF3FFF3FFF3FFF3FFF3F61
:100FA000FF3FFF3FFF3FFF3FFF3FFF3FFF3FFF3F51
:100FB000FF3FFF3FFF3FFF3FFF3FFF3FFF3FFF3F41
:100FC000FF3FFF3FFF3FFF3FFF3FFF3FFF3FFF3F31
:100FD000FF3FFF3FFF3FFF3FFF3FFF3FFF3FFF3F21
:100FE000FF3FFF3FFF3FFF3FFF3FFF3FFF3FFF3F11
:100FF000FF3FFF3FFF3FFF3FFF3FFF3FFF3FFF3F01
:101000006230A0006130A1007330A2007330A300F1
:101010005908193C031959285908183C0319632821
:101020005908173C031974285908163C03197E28DF
:101030005908153C03198F285908143C031997289F
:101040005908133C0319A6285908123C0319AE2865
:101050005908113C0319BD285908103C0319C5282B
:1010600059080F3C0319D42859080E3C0319D428F9
:1010700059080D3C0319DA2859080C3C0319E928D2
:1010800059080B3C0319F12859080A3C0319002997
:101090005908093C031908295908083C031917295C
:1010A0005908073C03191F295908063C0319302920
:1010B0003A292B30A8003130A9003530AA00FF3082
:1010C000BC00BD003A292B30A8003130A9003330D4
:1010D000AA002E30AB003530AC000030BB00FF3032
:1010E000BC000130BD003A292B30A8003130A900E6
:1010F0003230AA00FF30BB00BC003A292B30A800D8
:101100003130A9003030AA002E30AB003530AC00B1
:101110000030BA00FF30BB000130BC003A292B3050
:10112000A8003930AA00FF30BA00BB003A292B30A2
:10113000A8003730AA002E30AB003530AC000030AC
:10114000B900FF30BA000130BB003A292B30A800AB
:101150003630AA00FF30B900BA003A292B30A80077
:101160003430AA002E30AB003530AC000030B8006F
:10117000FF30B9000130BA003A292B30A8003330D3
:10118000AA00FF30B800B9003A292B30A80031304E
:10119000AA002E30AB003530AC000030B700FF3075
:1011A000B8000130B9003A293030AA00FF30B7004A
:1011B000B8003A29B030A8003130AA002E30AB0078
:1011C0003530AC000030B600FF30B7000130B80059
:1011D0003A29B030A8003330AA00FF30B600B7007B
:1011E0003A29B030A8003430AA002E30AB00353098
:1011F000AC000030B500FF30B6000130B7003A292E
:10120000B030A8003630AA00FF30B500B6003A2949
:10121000B030A8003730AA002E30AB003530AC001B
:101220000030B400FF30B5000130B6003A29B030CC
:10123000A8003930AA00FF30B400B5003A29B03018
:10124000A8003130A9003030AA002E30AB00353074
:10125000AC000030B300FF30B4000130B5003A29D3
:10126000B030A8003130A9003230AA00FF30B300FE
:10127000B4003A296430AE004230AF000800743048
:10128000A0007230A1006530A2006230A3006C3073
:10129000A4006530A5005A080A3C031970295A08B1
:1012A000093C03197A295A08083C031982295A086B
:1012B000073C03198A295A08063C031992295A083F
:1012C000053C031998295A08043C0319A0295A0817
:1012D000033C0319A8295A08023C0319B029BA296A
:1012E0002B30A8003130A9003230AA00FF30BB00FB
:1012F000BC00BA292B30A8003930AA00FF30BA0050
:10130000BB00BA292B30A8003630AA00FF30B90044
:10131000BA00BA292B30A8003330AA00FF30B80039
:10132000B900BA293030AA00FF30B700B800BA2996
:10133000B030A8003330AA00FF30B600B700BA2999
:10134000B030A8003630AA00FF30B500B600BA2988
:10135000B030A8003930AA00FF30B400B500BA2977
:10136000B030A8003130A9003230AA00FF30B300FD
:10137000B400BA296430AE004230AF000800DE1E6F
:10138000C229D7296230A0006130A1006C30A200D0
:101390006130A3006E30A4006330A5006530A60064
:1013A000B030AA006430AE004230AF00EC29B0305B
:1013B000A0006430A4004230A5006230A900613072
:1013C000AA006C30AB006130AC006E30AD00633011
:1013D000AE006530AF00EC295E08073C0319B52A62
:1013E0005E08083C0319BB2A5E08093C0319C32A9E
:1013F0005E080A3C0319CB2A5E080B3C0319D32A6A
:101400005E080C3C0319DD2A5E080D3C0319E72A2F
:101410005E080E3C0319F02A5E080F3C0319FB2AF4
:101420005E08103C0319062B5E08113C0319102BB3
:101430005E08123C03191C2B5E08133C0319282B71
:101440005E08143C0319332B5E08153C0319402B2E
:101450005E08163C03194D2B5E08173C0319572BE9
:101460005E08183C0319632B5E08193C03196F2BA7
:101470005E081A3C03197A2B5E081B3C0319872B64
:101480005E081C3C0319942B5E081D3C0319A02B1D
:101490005E081E3C0319AE2B5E081F3C0319BC2BD3
:1014A0005E08203C0319BD2B5E08213C0319E02B8C
:1014B0005E08223C0319EE2B5E08233C0319FC2B2B
:1014C0005E08243C0319092C5E08253C0319162CE0
:1014D0005E08263C0319232C5E08273C03192E2C9A
:1014E0005E08283C03193A2C5E08293C0319462C57
:1014F0005E082A3C0319502C5E082B3C03195D2C16
:101500005E082C3C03196A2C5E082D3C0319752CCF
:101510005E082E3C0319812C5E082F3C03198D2C8C
:101520005E08303C0319972C5E08313C0319A22C4D
:101530005E08323C0319AD2C5E08333C0319B62C0F
:101540005E08343C0319C02C5E08353C0319CA2CD4
:101550005E08363C0319D22C5E08373C0319DA2C9E
:101560005E08383C0319E22CE82C3830AB003030F0
:10157000AC00E924E82C3230AB003330AC00E92475
:101580000130B800E82C3230AB003230AC00E92436
:101590000430B800E82C3230AB003130AC00E92424
:1015A000FF30B800E82C3230AB003030AC00E9241A
:1015B000FF30B8000130B900E82C3130AB003930D1
:1015C000AC00E924FF30B8000430B900E82C313019
:1015D000AB003830AC00E924FF30B800B900E82C8B
:1015E0003130AB003730AC00E924FF30B800B9002F
:1015F0000130BA00E82C3130AB003630AC00E924C1
:10160000FF30B800B9000430BA00E82C3130AB002C
:101610003530AC00E924FF30B800B900BA00E82C3E
:101620003130AB003430AC00E924FF30B800B900F1
:10163000BA000130BB00E82C3130AB003330AC00D5
:10164000E924FF30B800B900BA000430BB00E82C30
:101650003130AB003230AC00E924FF30B800B900C3
:10166000BA00BB00E82C3130AB003130AC00E924CB
:10167000FF30B800B900BA00BB000130BC00E82C54
:101680003130AB003030AC00E924FF30B800B90095
:10169000BA00BB000430BC00E82C3930AC00E924AF
:1016A000FF30B800B900BA00BB00BC00E82C3830ED
:1016B000AC00E924FF30B800B900BA00BB00BC00A0
:1016C0000130BD00E82C3730AC00E924FF30B80011
:1016D000B900BA00BB00BC000430BD00E82C3630B5
:1016E000AC00E924FF30B800B900BA00BB00BC0070
:1016F000BD00E82C3530AC00E924FF30B800B9005B
:10170000BA00BB00BC00BD000130BE00E82C343084
:10171000AC00E924FF30B800B900BA00BB00BC003F
:10172000BD000430BE00E82C3330AC00E924FF30AB
:10173000B800B900BA00BB00BC00BD00BE00E82C78
:101740003230AC00E924FF30B800B900BA00BB0069
:10175000BC00BD00BE000130BF00E82C3130AC0041
:10176000E924FF30B800B900BA00BB00BC00BD00DE
:10177000BE000430BF00E82C0000FE30A000FE30A8
:10178000A100FE30A200FE30A300FE30A4006230B3
:10179000A5006130A6006C30A7006130A8006E3053
:1017A000A9006330AA006530AB00FE30AC00FE300B
:1017B000AD00FE30AE00FE30AF00FA24E924E82C84
:1017C0003130A200FA24FF30B700B600B500B400F3
:1017D000B300B200B1000530B000E82C3230A200F6
:1017E000FA24FF30B700B600B500B400B300B20071
:1017F000B1000030B000E82C3330A200FA24FF30F2
:10180000FF30B700B600B500B400B300B200B100BD
:10181000E82C3430A200FA24FF30B700B600B5003F
:10182000B400B300B2000530B100E82C3530A2009E
:10183000FA24FF30B700B600B500B400B300B20020
:101840000030B100E82C3630A200FA24FF30B70097
:10185000B600B500B400B300B200E82C3730A200E7
:10186000FA24FF30B700B600B500B400B30005306D
:10187000B200E82C3830A200FA24FF30B700B600DE
:10188000B500B400B3000030B200E82C3930A2003B
:10189000FA24FF30B700B600B500B400B300E82C5E
:1018A0003130A1003030A200FA24FF30B700B6007A
:1018B000B500B4000530B300E82C3130A100313060
:1018C000A200FA24FF30B700B600B500B400003023
:1018D000B300E82C3130A1003230A200FA24FF30EE
:1018E000B700B600B500B400E82C3130A1003330A9
:1018F000A200FA24FF30B700B600B5000530B400EE
:10190000E82C3130A1003430A200FA24FF30B700B7
:10191000B600B5000030B400E82C3130A1003530FD
:10192000A200FA24FF30B700B600B500E82C313031
:10193000A1003630A200FA24FF30B700B60005300F
:10194000B500E82C3130A1003730A200FA24FF3076
:10195000B700B6000030B500E82C3130A1003830B7
:10196000A200FA24FF30B700B600E82C3130A10005
:101970003930A200FA24FF30B7000530B600E82C59
:101980003230A1003030A200FA24FF30B70000301E
:10199000B600E82C3230A1003130A200FA24FF302A
:1019A000B700E82C3230A1003230A200FA24053012
:1019B000B700E82C3230A1003330A200FA24003006
:1019C000B700E82C3830A1003030A200FA24E82C0F
:1019D0000800FF30B000FF30B100FF30B200FF3030
:1019E000B300FF30B400FF30B500FF30B600FF3069
:1019F000B7000800FF30B800FF30B900FF30BA0070
:101A0000FF30BB00FF30BC00FF30BD00FF30BE0028
:101A1000FF30BF000800FF3FFF3FFF3FFF3FFF3F9A
:101A2000FF3FFF3FFF3FFF3FFF3FFF3FFF3FFF3FC6
:101A3000FF3FFF3FFF3FFF3FFF3FFF3FFF3FFF3FB6
:101A4000FF3FFF3FFF3FFF3FFF3FFF3FFF3FFF3FA6
:101A5000FF3FFF3FFF3FFF3FFF3FFF3FFF3FFF3F96
:102000007630A0006F30A1006C30A2007530A300C4
:102010006D30A4006530A50058083F3C0319ED2839
:1020200058083E3C0319052958083D3C03191E2950
:1020300058083C3C0319372958083B3C03195029E0
:1020400058083A3C031967295808393C03197F2975
:102050005808383C031995295808373C0319A92911
:102060005808363C0319BE295808353C0319D329B2
:102070005808343C0319E8295808333C0319FB2954
:102080005808323C03190F2A5808313C0319232AF7
:102090005808303C0319352A58082F3C0319462AA2
:1020A00058082E3C0319592A58082D3C03196A2A4E
:1020B00058082C3C03197B2A58082B3C03198D2AFD
:1020C00058082A3C03199F2A5808293C0319AF2AAB
:1020D0005808283C0319C02A5808273C0319D12A5C
:1020E0005808263C0319E02A5808253C0319F22A0F
:1020F0005808243C0319042B5808233C0319162BB9
:102100005808223C0319262B5808213C0319372B69
:102110005808203C0319482B58081F3C0319572B1B
:1021200058081E3C0319672B58081D3C0319772BD0
:1021300058081C3C0319872B58081B3C0319952B86
:1021400058081A3C0319A42B5808193C0319B32B3F
:102150005808183C0319C02B5808173C0319CE2BFC
:102160005808163C0319DC2B5808153C0319E82BBA
:102170005808143C0319F42B5808133C0319012C7C
:102180005808123C03190E2C5808113C0319192C3D
:102190005808103C03192B2C58080F3C0319372CF6
:1021A00058080E3C0319412C58080D3C03194C2CBF
:1021B00058080C3C0319572C58080B3C0319622C87
:1021C00058080A3C03196B2C5808093C0319742C55
:1021D0005808083C03197D2C842C2B30AA00313080
:1021E000AB003530AC00FF30B000B100B200B3003E
:1021F000B400B500B600B700B800B900BA00BB0023
:10220000BC00BD00BE00BF00842C2B30AA003130C2
:10221000AB003430AC00FF30B000B100B200B3000E
:10222000B400B500B600B700B800B900BA00BB00F2
:10223000BC00BD00BE000430BF00842C2B30AA00BF
:102240003130AB003330AC00FF30B000B100B20031
:10225000B300B400B500B600B700B800B900BA00CA
:10226000BB00BC00BD00BE000330BF00842C2B307F
:10227000AA003130AB003230AC00FF30B000B1000A
:10228000B200B300B400B500B600B700B800B900A2
:10229000BA00BB00BC00BD00BE000230BF00842CF1
:1022A0002B30AA003130AB003130AC00FF30B00031
:1022B000B100B200B300B400B500B600B700B8007A
:1022C000B900BA00BB00BC00BD00BE00842C2B309E
:1022D000AA003130AB003030AC00FF30B000B100AC
:1022E000B200B300B400B500B600B700B800B90042
:1022F000BA00BB00BC00BD000330BE00842C2B30F4
:10230000AA003930AC00FF30B000B100B200B30019
:10231000B400B500B600B700B800B900BA00BB0001
:10232000BC00BD000130BE00842C2B30AA00383028
:10233000AC00FF30B000B100B200B300B400B50093
:10234000B600B700B800B900BA00BB00BC00BD00C1
:10235000842C2B30AA003730AC00FF30B000B10025
:10236000B200B300B400B500B600B700B800B900C1
:10237000BA00BB00BC000430BD00842C2B30AA0086
:102380003630AC00FF30B000B100B200B300B40092
:10239000B500B600B700B800B900BA00BB00BC0079
:1023A0000130BD00842C2B30AA003530AC00FF304A
:1023B000B000B100B200B300B400B500B600B70081
:1023C000B800B900BA00BB00BC000230BD00842CCC
:1023D0002B30AA003430AC00FF30B000B100B200A6
:1023E000B300B400B500B600B700B800B900BA0039
:1023F000BB00BC00842C2B30AA003330AC00FF3073
:10240000B000B100B200B300B400B500B600B70030
:10241000B800B900BA00BB000330BC00842C2B30DC
:10242000AA003230AC00FF30B000B100B200B300FF
:10243000B400B500B600B700B800B900BA00BB00E0
:102440000230BC00842C2B30AA003130AC00FF30AD
:10245000B000B100B200B300B400B500B600B700E0
:10246000B800B900BA00BB00842C3030AC00FF309B
:10247000B000B100B200B300B400B500B600B700C0
:10248000B800B900BA000430BB00842CB030AA00F8
:102490003130AC00FF30B000B100B200B300B40086
:1024A000B500B600B700B800B900BA000130BB00F3
:1024B000842CB030AA003230AC00FF30B000B10044
:1024C000B200B300B400B500B600B700B800B90060
:1024D000BA00842CB030AA003330AC00FF30B0001A
:1024E000B100B200B300B400B500B600B700B80048
:1024F000B900BA00842CB030AA003430AC00FF30F0
:10250000B000B100B200B300B400B500B600B7002F
:10251000B800B9000330BA00842CB030AA003530BE
:10252000AC00FF30B000B100B200B300B400B500A1
:10253000B600B700B800B9000230BA00842CB03041
:10254000AA003630AC00FF30B000B100B200B300DA
:10255000B400B500B600B700B800B900842CB030A4
:10256000AA003730AC00FF30B000B100B200B300B9
:10257000B400B500B600B700B8000430B900842C30
:10258000B030AA003830AC00FF30B000B100B2006B
:10259000B300B400B500B600B700B8000130B90010
:1025A000842CB030AA003930AC00FF30B000B1004C
:1025B000B200B300B400B500B600B700B800842C78
:1025C000B030AA003130AB003030AC00FF30B0008A
:1025D000B100B200B300B400B500B600B7000430DB
:1025E000B800842CB030AA003130AB003130AC00E0
:1025F000FF30B000B100B200B300B400B500B600C7
:10260000B7000330B800842CB030AA003130AB00E2
:102610003230AC00FF30B000B100B200B300B40003
:10262000B500B600B7000230B800842CB030AA0064
:102630003130AB003330AC00FF30B000B100B2003D
:10264000B300B400B500B600B700842CB030AA00C7
:102650003130AB003430AC00FF30B000B100B2001C
:10266000B300B400B500B6000330B700842CB0301E
:10267000AA003130AB003530AC00FF30B000B10003
:10268000B200B300B400B500B6000130B700842C2E
:10269000B030AA003130AB003630AC00FF30B000B3
:1026A000B100B200B300B400B500B600842CB03065
:1026B000AA003130AB003730AC00FF30B000B100C1
:1026C000B200B300B400B5000430B600842CB030C2
:1026D000AA003130AB003830AC00FF30B000B100A0
:1026E000B200B300B400B5000130B600842CB030A5
:1026F000AA003130AB003930AC00FF30B000B1007F
:10270000B200B300B400B5000230B600842CB03083
:10271000AA003230AB003030AC00FF30B000B10066
:10272000B200B300B400B500842CB030AA0032303F
:10273000AB003130AC00FF30B000B100B200B300EC
:10274000B4000330B500842CB030AA003230AB00A6
:102750003230AC00FF30B000B100B200B300B400C2
:102760000230B500842CB030AA003230AB003330D8
:10277000AC00FF30B000B100B200B300B400842C54
:10278000B030AA003230AB003430AC00FF30B000C3
:10279000B100B200B3000430B400842CB030AA0001
:1027A0003230AB003530AC00FF30B000B100B200C9
:1027B000B3000130B400842CB030AA003230AB003A
:1027C0003630AC00FF30B000B100B200B300842C52
:1027D000B030AA003230AB003730AC00FF30B00070
:1027E000B100B200B300842CB030AA003230AB008C
:1027F0003830AC00FF30B000B100B2000330B3009D
:10280000842CB030AA003230AB003930AC00FF303D
:10281000B000B100B2000230B300842CB030AA0086
:102820003330AB003030AC00FF30B000B100B2004C
:10283000842CB030AA003330AB003130AC00B03063
:10284000AA003330AB003230AC00FF30B000B10032
:102850000430B200842CB030AA003330AB003230E8
:10286000AC00FF30B000B1000130B200842CB030B9
:10287000AA003330AB003330AC00FF30B000B10001
:10288000842CB030AA003330AB003430AC00FF30C1
:10289000B0000430B100842CB030AA003330AB005B
:1028A0003530AC00FF30B0000330B100842CB030C4
:1028B000AA003330AB003630AC00FF30B00002303D
:1028C000B100842CB030AA003330AB003730AC00FC
:1028D000FF30B000842CB030AA003330AB00383069
:1028E000AC000330B000842CB030AA003330AB0011
:1028F0003930AC000130B000842CB030AA00343044
:10290000AB003030AC00842C6430AE004230AF00FD
:102910000800FF3FFF3FFF3FFF3FFF3FFF3FFF3FFD
:10292000FF3FFF3FFF3FFF3FFF3FFF3FFF3FFF3FB7
:10293000FF3FFF3FFF3FFF3FFF3FFF3FFF3FFF3FA7
:10294000FF3FFF3FFF3FFF3FFF3FFF3FFF3FFF3F97
:10295000FF3FFF3FFF3FFF3FFF3FFF3FFF3FFF3F87
:10300000E31F8528E31363088207852886288C2818
:1030100093289B28A428AC28B628BF28CA28D528DE
:10302000DF28EB28F82804290F291C29292936290B
:1030300043294F295B2969297729852985299329DE
:10304000A029AD29AD29BC29CB29CB29DA29DA2938
:10305000E929E929F729F729052A052A152A152A30
:10306000252A252A352A352A452A452A452A542A39
:10307000542A632A632A632A742A742A742A852AA2
:10308000852A852A962A962A962AA72AA72AA72A2F
:10309000A72AB72AB72AB72AC72AC72AC72AC72AF8
:1030A000D92AD92AD92AD92AEB2AEB2AEB2AEB2AC0
:1030B000FD2AFD2AFD2AFD2A0F2B0F2B0F2B0F2B8C
:1030C0000F2B202B202B202B202B312B312B312B86
:1030D000312B312B442B442B442B442B442B442B9E
:1030E000572B572B572B572B572B6A2B6A2B6A2B97
:1030F0006A2B6A2B6A2B7D2B7D2B7D2B7D2B7D2BC9
:103100007D2B8F2B8F2B8F2B8F2BA12BFF30F00044
:10311000F1000130F200A12BFF30F000F100F200CD
:103120000430F300A12BFF30F000F100F200F300B7
:103130000330F400A12BFF30F000F100F200F300A7
:10314000F4000130F500A12BFF30F000F100F20097
:10315000F300F400F500A12BFF30F000F100F200C5
:10316000F300F400F5000430F600A12BFF30F0006E
:10317000F100F200F300F400F500F600A12BFF309F
:10318000F000F100F200F300F400F500F600023068
:10319000F700A12BFF30F000F100F200F300F40083
:1031A000F500F6000430F700A12BFF30F000F1002D
:1031B000F200F300F400F500F600F700A12BFF3059
:1031C000F000F100F200F300F400F500F600F70063
:1031D0000230F800A12BFF30FF30F000F100F200C8
:1031E000F300F400F500F600F7000330F800A12B1F
:1031F000FF30F000F100F200F300F400F500F600FB
:10320000F7000430F800A12BFF30F000F100F200CD
:10321000F300F400F500F600F700F800A12BFF30F2
:10322000F000F100F200F300F400F500F600F70002
:10323000F8000230F900A12BFF30F000F100F2009D
:10324000F300F400F500F600F700F8000130F90093
:10325000A12BFF30F000F100F200F300F400F500C4
:10326000F600F700F8000330F900A12BFF30F00062
:10327000F100F200F300F400F500F600F700F800AA
:103280000430F900A12BFF30F000F100F200F30050
:10329000F400F500F600F700F800F900A12BFF306C
:1032A000F000F100F200F300F400F500F600F70082
:1032B000F800F900A12BFF30F000F100F200F3005C
:1032C000F400F500F600F700F800F9000230FA000B
:1032D000A12BFF30F000F100F200F300F400F50044
:1032E000F600F700F800F9000130FA00A12BFF30DA
:1032F000F000F100F200F300F400F500F600F70032
:10330000F800F9000330FA00A12BFF30F000F100C3
:10331000F200F300F400F500F600F700F800F90001
:103320000430FA00A12BFF30F000F100F200F300AE
:10333000F400F500F600F700F800F900FA00A12B00
:10334000FF30F000F100F200F300F400F500F600A9
:10335000F700F800F900FA00A12BFF30F000F100AF
:10336000F200F300F400F500F600F700F800F900B1
:10337000FA000230FB00A12BFF30F000F100F20058
:10338000F300F400F500F600F700F800F900FA0089
:103390000130FB00A12BFF30F000F100F200F30040
:1033A000F400F500F600F700F800F900FA00033029
:1033B000FB00A12BFF30F000F100F200F300F4005D
:1033C000F500F600F700F800F900FA000430FB0001
:1033D000A12BFF30F000F100F200F300F400F50043
:1033E000F600F700F800F900FA00FB00A12BFF300F
:1033F000F000F100F200F300F400F500F600F70031
:10340000F800F900FA00FB00A12BFF30F000F100FA
:10341000F200F300F400F500F600F700F800F90000
:10342000FA00FB000230FC00A12BFF30F000F1009D
:10343000F200F300F400F500F600F700F800F900E0
:10344000FA00FB000130FC00A12BFF30F000F1007E
:10345000F200F300F400F500F600F700F800F900C0
:10346000FA00FB000330FC00A12BFF30F000F1005C
:10347000F200F300F400F500F600F700F800F900A0
:10348000FA00FB000430FC00A12BFF30F000F1003B
:10349000F200F300F400F500F600F700F800F90080
:1034A000FA00FB00FC00A12BFF30F000F100F2005D
:1034B000F300F400F500F600F700F800F900FA0058
:1034C000FB00FC00A12BFF30F000F100F200F30044
:1034D000F400F500F600F700F800F900FA00FB0030
:1034E000FC000230FD00A12BFF30F000F100F200E3
:1034F000F300F400F500F600F700F800F900FA0018
:10350000FB00FC000130FD00A12BFF30F000F100BA
:10351000F200F300F400F500F600F700F800F900FF
:10352000FA00FB00FC000330FD00A12BFF30F0008F
:10353000F100F200F300F400F500F600F700F800E7
:10354000F900FA00FB00FC000430FD00A12BFF3065
:10355000F000F100F200F300F400F500F600F700CF
:10356000F800F900FA00FB00FC00FD00A12BFF3081
:10357000F000F100F200F300F400F500F600F700AF
:10358000F800F900FA00FB00FC00FD00A12BFF3061
:10359000F000F100F200F300F400F500F600F7008F
:1035A000F800F900FA00FB00FC00FD000230FE000C
:1035B000A12BFF30F000F100F200F300F400F50061
:1035C000F600F700F800F900FA00FB00FC00FD002F
:1035D0000130FE00A12BFF30F000F100F200F300FB
:1035E000F400F500F600F700F800F900FA00FB001F
:1035F000FC00FD000330FE00A12BFF30F000F100C5
:10360000F200F300F400F500F600F700F800F9000E
:10361000FA00FB00FC00FD000430FE00A12BFF308F
:10362000F000F100F200F300F400F500F600F700FE
:10363000F800F900FA00FB00FC00FD00FE00A12BE1
:10364000FF30F000F100F200F300F400F500F600A6
:10365000F700F800F900FA00FB00FC00FD00FE0096
:10366000A12BFF30F000F100F200F300F400F500B0
:10367000F600F700F800F900FA00FB00FC00FD007E
:10368000FE000230FF00A12BFF30F000F100F2003D
:10369000F300F400F500F600F700F800F900FA0076
:1036A000FB00FC00FD00FE000130FF00A12BFF30FD
:1036B000F000F100F200F300F400F500F600F7006E
:1036C000F800F900FA00FB00FC00FD00FE000330EA
:1036D000FF00A12BFF30F000F100F200F300F40036
:1036E000F500F600F700F800F900FA00FB00FC0016
:1036F000FD00FE000430FF00A12BFF30F000F100C0
:10370000F200F300F400F500F600F700F800F9000D
:10371000FA00FB00FC00FD00FE00FF00A12BFF30C3
:10372000F000F100F200F300F400F500F600F700FD
:10373000F800F900FA00FB00FC00FD00FE00FF00AD
:10374000A12B0800FF3FFF3FFF3FFF3FFF3FFF3F31
:10375000FF3FFF3FFF3FFF3FFF3FFF3FFF3FFF3F79
:10376000FF3FFF3FFF3FFF3FFF3FFF3FFF3FFF3F69
:10377000FF3FFF3FFF3FFF3FFF3FFF3FFF3FFF3F59
:10378000FF3FFF3FFF3FFF3FFF3FFF3FFF3FFF3F49
:1042000030000E0006001F001800FF00FF00FF0036
:10421000FF00FF00FF00FF00FF00FF00FF00FF00A6
:10422000FF00FF00FF00FF00FF00FF00FF00FF0096
:10423000FF00FF00FF00FF00FF00FF00FF00FF0086
:10424000FF00FF00FF00FF00FF00FF00FF00FF0076
:10425000FF00FF00FF00FF00FF00FF00FF00FF0066
:10426000FF00FF00FF00FF00FF00FF00FF00FF0056
:10427000FF00FF00FF00FF00FF00FF00FF00FF0046
:10428000FF00FF00FF00FF00FF00FF00FF00FF0036
:10429000FF00FF00FF00FF00FF00FF00FF00FF0026
:1042A000FF00FF00FF00FF00FF00FF00FF00FF0016
:1042B000FF00FF00FF00FF00FF00FF00FF00FF0006
:1042C000FF00FF00FF00FF00FF00FF00FF00FF00F6
:1042D000FF00FF00FF00FF00FF00FF00FF00FF00E6
:1042E000FF00FF00FF00FF00FF00FF00FF00FF00D6
:1042F000FF00FF00FF00FF00FF00FF00FF00FF00C6
:10430000FF00FF00FF00FF00FF00FF00FF00FF00B5
:10431000FF00FF00FF00FF00FF00FF00FF00FF00A5
:10432000FF00FF00FF00FF00FF00FF00FF00FF0095
:10433000FF00FF00FF00FF00FF00FF00FF00FF0085
:10434000FF00FF00FF00FF00FF00FF00FF00FF0075
:10435000FF00FF00FF00FF00FF00FF00FF00FF0065
:10436000FF00FF00FF00FF00FF00FF00FF00FF0055
:10437000FF00FF00FF00FF00FF00FF00FF00FF0045
:10438000FF00FF00FF00FF00FF00FF00FF00FF0035
:10439000FF00FF00FF00FF00FF00FF00FF00FF0025
:1043A000FF00FF00FF00FF00FF00FF00FF00FF0015
:1043B000FF00FF00FF00FF00FF00FF00FF00FF0005
:1043C000FF00FF00FF00FF00FF00FF00FF00FF00F5
:1043D000FF00FF00FF00FF00FF00FF00FF00FF00E5
:1043E000FF00FF00FF00FF00FF00FF00FF00FF00D5
:1043F000FF00FF00FF00FF00FF00FF00FF00FF00C5
:04400E00FD2FFF3F44
:08400000FF3FFF3FFF3FFF3FC0
:00000001FF
